:10000000830100308A002D28F00003088301E600F8
:100010000408E7000A08E8008A016908EB006A089A
:10002000EC0083160C1E182883120C1E18285E2361
:1000300083168C1E1F2883128C1E1F28AE2383124A
:100040006B08E9006C08EA006708840068088A0009
:1000500066088300F00E700E0900203084006630C0
:100060003A20A0308400E2303A2083013A2B040683
:100070008001840A0406031D372800348312E90036
:10008000EA1B49286A088A006908E90A0319EA0A8A
:10009000820083136A1883176908E90A840000083C
:1000A0000800820730343134323433343434353458
:1000B0003634373438343934613462346334643438
:0400C0006534663409
:10065A000D3071230A30712B831265085023640808
:10066A005023630850236208502B073083129F00DF
:10067A008B17C82343238423E323402B8316861333
:10068A0006138612861185110511851005100610AC
:10069A008312061408008312E20000308A00620EF8
:1006AA000F395120712300308A0062080F39512016
:1006BA00712B8312200803196B2B2108223E840018
:1006CA0000089900210A3F39A100A00320088316D7
:1006DA0003190C12831208008312E2008312201BF2
:1006EA00732B8B13210820073F39223E84006208AE
:1006FA008000A00A83160C168B1783120800831633
:10070A0020080319842B2108A23E840000088312C2
:10071A00E2008B138316210A3F39A100A0038B172D
:10072A00831262080800A12B6308EA006208E20A41
:10073A000319E30A3E207123831263086204031932
:10074A0008006308EA0062083E200038031908001E
:10075A00992B83121819C52B981CB62B1812181628
:10076A00C62B8316201BC42B210820073F39A23E23
:10077A00840083121A0880008316A00AC62B8312EB
:10078A001A08831208008312A001A1018316A0018E
:10079A00A10186140615181519309900181283122A
:1007AA00981718169812831618138312181383169B
:1007BA0098160C128C160B17831208008312E2008B
:1007CA008613E21B86170613621B06178612E21AA5
:1007DA0086168611621A86158511E2198515051184
:1007EA00621905158510E21885140510621805149A
:0607FA00061006140800C1
:02400E00F03F81
:00000001FF
